:10000000023F61FFFFFFFFFFFFFFFF0239FBFFFF22
:10001000FFFFFFFFFFFFFFFFFFFFFF02376CFFFF48
:10002000FFFFFFFFFFFFFFFFFFFFFFD227C2C63228
:10005000FFFFFF024296FFFFFFFFFF0242FFFFFF8D
:10006000FFFFFFFFFFFFFFFFFFFFFF0230EDFFFF7E
:10007000FFB050FFFFFFFFFFFFFFFFFFFFFFFFFF8E
:10008000FFFFFFFFFFFFFFFFFFFFFF024004FFFF37
:1001000078D976FFC2E9C2EAC2EB900005E4F0A319
:10011000F090000474FFF0758680D2AED2BE78866F
:10012000F6E6F8E4F678E4F678F4F208F278A8F265
:1001300008F278F6F208F278F4E2FE08E2F5828E30
:1001400083E493FE740193FF78A9E22FF218E23E54
:10015000F278F5E22402F218E23400F278F7E224B1
:1001600001F218E23400F208E2B400CB18E2B44025
:10017000C6900002801078A9E2700218E2600ED2E8
:10018000EBD2EA9000057455F0A3F080E9C2AFE429
:10019000F5A8F5B8758680C28C438911758CF27507
:1001A0008AFAD28C12411F759A02D2A9D2ABC2CF61
:1001B000C2CED2CCD2CBC2CAC2C9D2C875C150C27B
:1001C000C5C2C4C2C3C2C6C2BFD2AD12444F75516C
:1001D000FFD28875A93075B93CE4F55B90000474D2
:1001E000FFF0F5F8E478D6F678CC76FF7880F678EC
:1001F0008D76FFFE7F087D04FB7A00796F124482C2
:100200007E007F087DFF7BFE7AF879D012448278E9
:10021000AC7482F2787D7488F278D8760178CD76E5
:10022000FF900005E4F0A3F0900000F0A3F0A374A9
:1002300055F0A3F0E4F55FC2EBC2E9C2EAC29578DB
:10024000CFF2787C7428F2D2AF7DC57B027F7E121C
:100250004399400CC2AF90000474FFF0D2E980F4DF
:1002600078C576550876AA787B74AAF278977402D6
:10027000F2788C7481F27DC57B027F7E12421C5025
:10028000D3E4788CF27F641244B27DC77B027F7E18
:1002900012439950BF79C5E778C766700609E70829
:1002A000666004D2EA80AD7DC57B017F061243996A
:1002B0007F051244B27DC67B017F071243997F05FB
:1002C0001244B27DC77B017F081243997F05124417
:1002D000B27DC87B017F091243997F051244B27D2C
:1002E000C97B017F0A12439978C5E678CAF678C6B9
:1002F000E66417600302042C08E664046003020449
:100300002C08E664AA600302042C08E66455600326
:1003100002042C08E6C39440400302042C78C576FE
:1003200018787B74E7F27DC57B017F07123ECE7F94
:100330000A1244B278C57605787B74FAF27DC57BE3
:10034000017F08123ECE7F0A1244B278C5765578F6
:100350007B74AAF27DC57B017F09123ECE7F0A1213
:1003600044B278C576AA787B7455F27DC57B017F4F
:100370000A123ECE7F0A1244B2123EBC7F0A1244D9
:10038000B2E4F55BE478C5F6787B74FFF2E55B24B4
:100390000BFF7DC57B01123ECE7F0A1244B2E4788A
:1003A000C5F6787B74FFF2E55B241EFF7DC57B01FB
:1003B000123ECE7F0A1244B2055BE55BC39408404F
:1003C000C3E4F55BE478C5F6787B74FFF2E55B2463
:1003D00013FF7DC57B01123ECE7F0A1244B2055B3E
:1003E000E55BC3940840DD78C57682787B747DF246
:1003F0007DC57B017F1B123ECE7F0A1244B278C5B9
:100400007688787B7477F27DC57B017F1C123ECEA7
:100410007F0A1244B278C57601787B74FEF27DC5FE
:100420007B017F1D123ECE7F0A1244B27D017F0602
:10043000123D077F051244B278C0E6900005F078BF
:10044000CAF6A3741AF07FF41244B278B376FF7D33
:10045000047F07123D0778C0E6B4181708E6B40514
:100460001208E6B4550D08E6B4AA0878CAE6C394A3
:10047000404072D23CC23478CAE6900005F0740461
:100480001244AE78C0E6900005F074081244AE78CD
:10049000C1E6900005F0A37410F07F641244B278B6
:1004A000C2E6900005F0A37420F07F641244B27895
:1004B000C3E6900005F0A37440F07F641244B27864
:1004C0007B7601E478CAF6FE7F08FD7BFE7AF87938
:1004D0000D12448278AC7482F2787D7488F278D8F8
:1004E0007601020593E4F55B755801E55BC394085A
:1004F000506DE55B240B123D0478C0E6FF740D25BA
:100500005BF8EFF2E55B241E123D0478C0E6B4FF11
:1005100002E4F678C0E6FF748F255BF8EFF2E55B46
:100520002413FF7D01123D0778C0E6F4F6E408F6D7
:1005300008760178C1E6FFC39408501979C0E7082E
:1005400056600874AB2FF8E55846F678C10608E601
:1005500025E0F680DE055BE55825E0F558808C7DCA
:10056000017F1B123D0778C0E678ACF27D017F1C4D
:10057000123D0778C0E6787DF27D017F1D123D07B0
:1005800078C0E678D8F67D017F26123D0778C0E670
:1005900078CFF278CAE6FF44C078C0F6EF60030275
:1005A000070F78C376FF1876FF78C576FF1876FFB9
:1005B000F5FA900000E0FFF531A3E0FEF532A3E08C
:1005C000FDF533A3E0FCF534E53130E30C78C2E609
:1005D00054FEF678C4E654FDF6E53130E70C78C2F7
:1005E000E654FBF678C4E654F7F6E53230E30C78CF
:1005F000C2E654EFF678C4E654DFF6E53230E70C95
:1006000078C2E654BFF678C4E6547FF6E53330E3AB
:100610000C78C3E654FEF678C5E654FDF6E53330B3
:10062000E70C78C3E654FBF678C5E654F7F6E534F4
:1006300030E30C78C3E654EFF678C5E654DFF6E510
:100640003430E70C78C3E654BFF678C5E6547FF63D
:1006500075FA018F318E328D338C34E53120E30C05
:1006600078C2E654FEF678C4E654FDF6E53120E79C
:100670000C78C2E654FBF678C4E654F7F6E532206F
:10068000E30C78C2E654EFF678C4E654DFF6E532C0
:1006900020E70C78C2E654BFF678C4E6547FF6E54E
:1006A0003320E30C78C3E654FEF678C5E654FDF635
:1006B000E53320E70C78C3E654FBF678C5E654F73B
:1006C000F6E53420E30C78C3E654EFF678C5E6543B
:1006D000DFF6E53420E70C78C3E654BFF678C5E6CC
:1006E000547FF6E4F55B78C2E6900005F008E6A3D7
:1006F000F07F0A1244B278C4E6900005F008E6A341
:10070000F07F0A1244B2055BE55BC3940F40D790BB
:100710000007E4F078E1F278D5F678C3F678D5E60C
:10072000FFC3940440030207DE780CE2FE9000054C
:10073000F07815E2FDA3F0900000EEF0A3EDF0EFED
:1007400014601014601B14602224037021780C7450
:1007500001800B780CE225E0F27013781504F2802A
:100760000A7815E225E0F27005800078D5067F163C
:100770001244B2E53A644670A478C3067816E2786B
:10078000C6F67817E278C7F67818E278C8F67819CE
:10079000E278C9F608E644C079C0F778C1764878AF
:1007A000E1E278C2F6E478C4F608F61241A4E4F572
:1007B0005F755B0179C6E778C74608460846555B12
:1007C000600678E1E2455BF2055FE55B25E0F55BFD
:1007D00070E278E1E27808F2753AFE02071D78CA05
:1007E000E644C079C0F778C1764378E1E278C2F692
:1007F000E478C4F61241A478CAE6FF1244B2E47861
:10080000D5F6F55F900005E52EF0A3E530F0E52E76
:10081000545525E0F55BE52E54AAC313425B9000C6
:1008200000E55BF0E530545525E0F55BE53054AA72
:10083000FFC313425BA3E55BF0755CFF753601E413
:10084000F550202F3F303204C232055F78E2E2607B
:100850000312273378CAE62464FFE433FEE55FB56C
:100860000713E4B5060FF55F78C0764508760108F2
:10087000760B1241A43042CAC242C2AFD2AED2BE3F
:10088000D2AF80BE78ACE26003B4FF1A78AC748259
:10089000F278C5F6F4787BF27DC57B017F1B123EB2
:1008A000CE7F0A1244B2787DE26003B4FF1A787DED
:1008B0007488F278C5F6F4787BF27DC57B017F1CE5
:1008C000123ECE7F0A1244B278D8E66003B4FF1C11
:1008D00078D8760178C576017401F4787BF27DC50D
:1008E0007B017F1D123ECE7F0A1244B2E478BFF630
:1008F000303602D2BD303902D2BA78E4E670030253
:100900000991C2AFB2EBB2E99000067403F0900017
:100910000574FFF0E478F6F208F278F6E2FE08E2F9
:10092000FFC394B8EE940B50218F828E83E493FE24
:10093000740193FF78A9E22FF218E23EF278F7E211
:100940002401F218E23400F280D0D2AED2BE900080
:1009500005E4F0A3F078F6F208F278F6E2FE08E299
:10096000FFC394B8EE940B50218F828E83E493FEE4
:10097000740193FF78A9E22FF218E23EF278F7E2D1
:100980002401F218E23400F280D0D2AED2BE0209C5
:10099000027886E6F8E67003020A2AC2AFB2EBB22A
:1009A000E990000674C0F090000574FFF0E478F65A
:1009B000F208F278F6E2FE08E2FFC394B8EE940B78
:1009C00050218F828E83E493FE740193FF78A9E215
:1009D0002FF218E23EF278F7E22401F218E2340036
:1009E000F280D0D2AED2BE900005E4F0A3F078F64B
:1009F000F208F278F6E2FE08E2FFC394B8EE940B38
:100A000050218F828E83E493FE740193FF78A9E2D4
:100A10002FF218E23EF278F7E22401F218E23400F5
:100A2000F280D0D2AED2BE02099B78A9E270021841
:100A3000E27003020AC3C2AFB2EBB2E9900005E56F
:100A40002EF0A374FFF0E478F6F208F278F6E2FEF6
:100A500008E2FFC394B8EE940B50218F828E83E49A
:100A600093FE740193FF78A9E22FF218E23EF27828
:100A7000F7E22401F218E23400F280D0D2AED2BE06
:100A8000900005E4F0A3F078F6F208F278F6E2FEC2
:100A900008E2FFC394B8EE940B50218F828E83E45A
:100AA00093FE740193FF78A9E22FF218E23EF278E8
:100AB000F7E22401F218E23400F280D0D2AED2BEC6
:100AC000020A2A208E05302A02D28E303068C230C7
:100AD000787BE2F4FF78CEE2FE6F705878C5A60608
:100AE00078D8E2FF7DC57B01123ECE7F0A1244B268
:100AF00078D8E26406703D78CEE27030D2AED2BED5
:100B0000F561E478C5F6787B74FFF278977401F2AA
:100B1000E561F4788CF27DC57B01AF6112421C5017
:100B2000F50561E561C3948040D880FE78CEE27817
:100B3000CAF6D223D229302926C22978D8E2FF7DED
:100B400001123D0778C0E678C3F678CDE278C2F6A8
:100B500078CAE644C079C0F778C176421241A42031
:100B60002303020C7FC22378C57618787B74E7F2E2
:100B70007DC57B017F07123ECE7F0A1244B278C545
:100B80007605787B74FAF27DC57B017F08123ECE34
:100B90007F0A1244B278C57655787B74AAF27DC577
:100BA0007B017F09123ECE7F0A1244B278C576AA35
:100BB000787B7455F27DC57B017F0A123ECE7F0A99
:100BC0001244B2123EBC203C03020C78E4F55B7484
:100BD0000D255BF8E278C5F6F4787BF2E55B240B33
:100BE000FF7DC57B01123ECE7F0A1244B2748F2571
:100BF0005BF8E278C5F6F4787BF2E55B241EFF7DB6
:100C0000C57B01123ECE7F0A1244B2E478C5F67865
:100C10007B74FFF2E55B2413FF7DC57B01123ECEA2
:100C20007F0A1244B2055BE55BC3940840A178AC2F
:100C3000E278C5F6F4787BF27DC57B017F1B123E1E
:100C4000CE7F0A1244B2787DE278C5F6F4787BF262
:100C50007DC57B017F1C123ECE7F0A1244B278D83C
:100C6000E6FF78C5F6EFF4787BF27DC57B017F1D4A
:100C7000123ECE7F0A1244B2C23CD2340202A7789E
:100C8000CDE6FFF4604690F711E054306420603CFC
:100C900078CAE644C079C0F778C1762808A60778F4
:100CA000CEE678C3F678CFE678C4F678D0E678C595
:100CB000F678D1E678C6F678D2E678C7F678D3E645
:100CC00078C8F678D41241A078CD76FF203203029E
:100CD000142BC232055F7883E2FF7886F2C3E55EAB
:100CE0009FF561C36480947850057561F8800CD3DA
:100CF000E561648094884003756108AF61EF3395C6
:100D0000E0FE7884E22FF218E23EF2787DE2047889
:100D10009AF67886E224CFF56178ACE224CEFFE43F
:100D200034FFFEAD61ED3395E0FCEF2DFFEE3CFEB0
:100D300078F6F208EFF2EE6004D2458002C2457800
:100D4000F7E278D7F630391A202503304803E4F566
:100D50002C302805E4F52CC228052CE52CB419020A
:100D6000C24130361E204803304403753514302DFF
:100D70000D303905753514800375350AC22DD5350A
:100D800002C23B303603303B06303909204106D2DF
:100D90002E78D57628203603303B0E303603303B94
:100DA00008303903304102C22EE55F540F706B7872
:100DB0008AE26005E214F2800F78CAE644C079C086
:100DC000F7E478C1F61241A4787CE2604DE214F2B7
:100DD000704878D5E66007787C7401F2803CE4F5D1
:100DE0005B746F255BF8E664047026740D255BF870
:100DF000E2FFD39407501A746F255BF8A607E55BF2
:100E0000901B6493425C78CFE2D394004003123B82
:100E100081055BE55BC3940840C730482690000419
:100E200074FFF0E47882F618F6787EF618F6787A91
:100E3000F618F618F618F6FE7F08FDFB7A00799290
:100E4000124482E55F54037052D235202E033044A1
:100E50004AE4F55175F8FF302E0890000474FFF055
:100E6000803978CCE6F4900004F0C28C758CFB7568
:100E70008AD5D28C3032FDC232D22C900000E0F400
:100E80007877F6A3E0F408F6A3E0F408F6A3E0F41C
:100E900008F675F8FF78D6E6F4A3F0E55F30E42FA6
:100EA000900005E52EF0A3E530F030345AE52E54DD
:100EB0005525E0F55BE52E54AAC313425B90000074
:100EC000E55BF0E530545525E0F55BE530802D908D
:100ED0000005E537F0A3E539F030342BE5375455FC
:100EE00025E0F55BE53754AAC313425B900000E5AB
:100EF0005BF0E539545525E0F55BE53954AAFFC3AD
:100F000013425BA3E55BF0303C33E55F7008900073
:100F10000574FFF0A3F0E55F541FFF7013787BE6C4
:100F2000900002F0F4A3F0E6FE25E0F670027601F0
:100F3000BF100A787BE6900000F0F4A3F0E55F3084
:100F4000E604C2EB8002D2EB78B5E66005D2EA1681
:100F50008002C2EA78D5E66013E55F30E404C2EAB5
:100F60008002D2EA202E1178D516800C78B4E66083
:100F700005D2E9168002C2E9304404D2EAD2E97807
:100F8000D9E66001167880E2A2E1506778D9E67070
:100F90006278CAE644C079C0F778C1764878CBE673
:100FA00006F8E678C2F678CBE606F8E678C3F67877
:100FB000CBE606F8E678C4F678CBE606F8E678C520
:100FC000F678CBE606F8E678C6F678CBE606F8E6DD
:100FD00078C7F678CBE606F8E678C8F678CBE6066A
:100FE000F81241A078D9761478CBE670067880E2C2
:100FF00054FDF27880E2A2E2506B78D9E670667810
:10100000CAE644C079C0F778C1764878CBE606F8DE
:10101000E278C2F678CBE606F8E278C3F678CBE65B
:1010200006F8E278C4F678CBE606F8E278C5F678FA
:10103000CBE606F8E278C6F678CBE606F8E278C7A3
:10104000F678CBE606F8E278C8F678CBE606F8E262
:1010500078C9F61241A478D9761478CBE670067870
:1010600080E254FBF27880E2A2E4503778D9E6704F
:101070003278CAE644C079C0F778C1764878CBE6C2
:10108000FF7DC27B0812439978CB740826F6124183
:10109000A478D9761478CBE6C3948040067880E2B1
:1010A00054EFF2E55C700302135878D9E66003024E
:1010B0001358E53625E0F53605506007E550D39422
:1010C000074006753601E4F550E55C553660D47589
:1010D0005B80E55555366003435B40E5215536603E
:1010E0000B435B087809E24536F2800B7809E2FF92
:1010F000E536F4FEEF5EF2E5225536600B435B10F9
:10110000780AE24536F2800B780AE2FFE536F4FE13
:10111000EF5EF2E5565536600B435B20780BE245F7
:1011200036F2800B780BE2FFE536F4FEEF5EF278E4
:10113000C2A65008A65B746F2550F8E678C4F6E5A1
:101140002FB55004E64410F6E5502408FFE433FEC2
:10115000E52FB5070AE4B5060678C4E64420F6781C
:10116000CD76FF74D92550F8E2700302132EE55BAB
:101170005418706BAF501244FE74D92550F8E4F245
:10118000E55025E025E024B0F8E4F2E55025E0251F
:10119000E024AFF8E4F2E55025E025E024AEF8E4E1
:1011A000F2E55025E025E024ADF8E4F2E55025E035
:1011B00025E0245DF8E4F2E55025E025E0245CF824
:1011C000E4F2E55025E025E0245BF8E4F2E5502563
:1011D000E025E0245AF8E4F278C176230213427441
:1011E000D92550F8E278C346F678C17627E478C866
:1011F000F618F618F618F678D0F618F618F678D429
:10120000F618F618F618F6755B05E55025E025E0AA
:10121000245AF8E2543FF560601378CDA65008A632
:1012200060E55025E025E024ADF8E28019E5502581
:10123000E025E024ADF8E2F560600EFFAE5B055BF3
:1012400074C02EF8EFF678D1F6E55025E025E024BD
:101250005BF8E2543FF560601478CDA65078CFA6D5
:1012600060E55025E025E024AEF8E28019E5502540
:10127000E025E024AEF8E2F560600EFFAE5B055BB2
:1012800074C02EF8EFF678D2F6E55025E025E0247C
:101290005CF8E2543FF560601478CDA65078D0A693
:1012A00060E55025E025E024AFF8E28019E55025FF
:1012B000E025E024AFF8E2F560600EFFAE5B055B71
:1012C00074C02EF8EFF678D3F6E55025E025E0243B
:1012D0005DF8E2543FF560603778CDA650E56025B3
:1012E000E025E0F56054C00846F6E56025E025E01D
:1012F000F56054C00846F6E56025E025E0F5605449
:10130000C00846F6E55025E025E024B0F8E2801953
:10131000E55025E025E024B0F8E2F5606024FFAE5A
:101320005B055B74C02EF8EFF678D4F6801478C1B4
:101330007623E55B5418AF5060051243DE8003123C
:1013400044FE78CAE644C079C0F71241A478D93087
:10135000440476648002760AE55F540778C6F6E6B0
:10136000240DF8E278C9F6C39464500302142B7478
:101370009C26F6E6C39403400302142BE55F30E29B
:1013800008900005E018F68007900004E078C8F6A1
:10139000E478C7F6E55F5403FF78C7E6C39F500BB8
:1013A00008E61313543FF6180680E978C8E654039C
:1013B000FFF678C6E6FE24D0F8E26F606E78C8E6E5
:1013C000FF74D02EF8EFF278C9E675F004A42FF57B
:1013D00082E435F0F583E582246CF582E583341BE5
:1013E000F583E493FF78C7F618E6246FF8E66F609C
:1013F0003A78C7E6FFB4041D18E6FE246FF8E4F659
:1014000074002EF8E4F274402EF582E434F9F5838A
:10141000740AF0801678C6E6FE246FF8EFF67400C2
:101420002EF8EFF2EE901B6493425C203503021815
:1014300038304803021838C2357562F9756340E4E4
:10144000F561E561C39408504E856382856283E04F
:101450006039E014F0E07033746F2561F87604743D
:10146000002561F87404F2AF617401A807088002D6
:10147000C333D8FC425C740D2561F8E2C394645018
:101480000A78CFE294004003123B8105610563E5D1
:101490006370AF056280AB302E030216C0122E952A
:1014A0008F61E561600302152E7D777B2E756737AE
:1014B000756801756902756A01FF1233817D7712C3
:1014C00033717D787B2E7567377568107569207567
:1014D0006A047F021233817D787B2E7567377568C9
:1014E00040756980756A087F031233817D797B308E
:1014F000756739756801756902756A107F04123362
:10150000817D797B30756739756804756908756AFE
:10151000207F051233817D7A7B30756739756810BD
:10152000756920756A407F061233810216A5E5575A
:1015300030E0065401553B6029E56F6404600AE51C
:1015400056455720E0033026047D7780027D7D7B61
:101550002E756737756801756902756A01E4FF12B7
:101560003381E55730E1065402553B6019E570645C
:1015700004600AE556455720E1033026047D778054
:10158000027D7D123371E55730E2065404553B600D
:1015900029E5716404600AE556455720E2033026C8
:1015A000047D7880027D7E7B2E75673775681075A7
:1015B0006920756A047F02123381E55730E30654CF
:1015C00008553B6029E5726404600AE556455720DA
:1015D000E3033026047D7880027D7E7B2E7567379D
:1015E000756840756980756A087F03123381E55715
:1015F00030E4065410553B6029E5736404600AE545
:1016000056455720E4033026047D7980027D817B96
:1016100030756739756801756902756A107F041243
:101620003381E55730E5065420553B6029E5746465
:1016300004600AE556455720E5033026047D79808D
:10164000027D817B30756739756804756908756A34
:10165000207F05123381E55730E6065440553B6044
:1016600029E5756404600AE556455720E6033026EF
:10167000047D7A80027D827B3075673975681075CC
:101680006920756A407F06123381E55730E70654BA
:1016900080553B6029E5766404600AE5564557208D
:1016A000E7033026047D7A80027D827B30756739BE
:1016B000756840756980756A807F07123381C2261C
:1016C000E4F55B755801E55BC394084003021838E4
:1016D000E55655586014E558F4FF78D656F67880EC
:1016E000E65FF678CCE65F02180A78CCE64558F655
:1016F0007883E64558F6746F255BF8E6B408004039
:101700000302182D90170BF82828730217430217AD
:10171000B40217670217230218030217D902178EA3
:1017200002173078D6E64558F67887E64558800C9B
:1017300078D6E64558F6E558F4788756F608E64533
:1017400058803578D6E64558F6E558F4FF78875640
:10175000F608E65FF608E65FF608E65FF608E65F7D
:10176000F608E65F0217FB78D6E64558F6E558F42A
:10177000FF788756F608E65FF608E64558F608E66D
:101780004558F608E64558F608E64558806D78D67F
:10179000E64558F6E558F4FF788756F608E65FF612
:1017A00008E65FF608E64558F608E64558F608E606
:1017B0004558804778D6E64558F6E558F4FF7887CF
:1017C00056F608E65FF608E65FF608E65FF608E616
:1017D0004558F608E64558802278D6E64558F6E59D
:1017E00058F4FF788756F608E65FF608E65FF608D5
:1017F000E65FF608E65FF608E64558F608E645585F
:10180000F6802AE558F4FF78D656F67887E65FF634
:1018100008E65FF608E65FF608E65FF608E65FF6BC
:1018200008E65FF608E65FF67883E65FF6055BE5B7
:101830005825E0F5580216C630437B204878C2434D
:10184000E4F55B755801E55BC394085069E55655AE
:10185000587059746F255BF8E6B40800504E901824
:1018600065F828287302187D02188D021881021865
:101870007F0218A502188D02188102187F80268029
:101880001C787FE6C394025002800A8010787FE6BD
:10189000C394035008E558F40856F6800F7880E6A4
:1018A0004558F68007E558F4788056F6055BE5580C
:1018B00025E0F558809078E2E26003122733E53A9C
:1018C00064466003021B49FF7E01EE7003021B4663
:1018D00078E1E25E6003021B3E7816E278C6F67895
:1018E00017E278C7F67818E278C8F67819E2FD783A
:1018F000C9F679C6E778C74608464D5E6003021B05
:101900003E756004E478C6F6F55BAD60056074165C
:101910002DF8E25E600AE55B901B649378C646F69C
:10192000055BE55BB408E3E478C2F6F55BAD600502
:101930006074162DF8E25E600AE55B901B64937894
:10194000C246F6055BE55BB406E305600560E47836
:10195000C7F6F55BAD60056074162DF8E25E600AAF
:10196000E55B901B649378C746F6055BE55BB408BE
:10197000E3E478C3F6F55BAD60056074162DF8E21C
:101980005E600AE55B901B649378C346F6055BE5F1
:101990005BB406E305600560E478C8F6F55BAD600E
:1019A000056074162DF8E25E600AE55B901B649397
:1019B00078C846F6055BE55BB408E3E478C4F6F561
:1019C0005BAD60056074162DF8E25E600AE55B9021
:1019D0001B649378C446F6055BE55BB406E30560DB
:1019E0000560E478C9F6F55BAD60056074162DF806
:1019F000E25E600AE55B901B649378C946F6055B7E
:101A0000E55BB408E3E478C5F6F55BAD60056074AA
:101A1000162DF8E25E600AE55B901B649378C5467C
:101A2000F6055BE55BB406E3EF25E025E024ADF8C1
:101A3000E278C6667067EF25E025E024AEF8E2782C
:101A4000C7667059EF25E025E024AFF8E278C86654
:101A5000704BEF25E025E024B0F8E278C966703DD0
:101A6000EF25E025E0245AF8E278C266702FEF25D2
:101A7000E025E0245BF8E278C3667021EF25E025DD
:101A8000E0245CF8E2FD78C4E6B50511EF25E02519
:101A9000E0245DF8E278C5667003021B3EE4F55B66
:101AA00078C6E6FD700578C2E66002055B78C7E699
:101AB000F9700578C3E66002055B78C8E6FC70053E
:101AC00078C4E66002055B78C9E6FB700578C5E678
:101AD0006002055BEF25E025E024ADF8EDF2EF258F
:101AE000E025E024AEF8E9F2EF25E025E024AFF8A8
:101AF000ECF2EF25E025E024B0F8EBF278C2E6FD49
:101B0000EF25E025E0245AF8EDF278C3E6FDEF2555
:101B1000E025E0245BF8EDF278C4E6FDEF25E02552
:101B2000E0245CF8EDF278C5E6FDEF25E025E02441
:101B30005DF8EDF274D92FF8E55BF2EE425C0FEE42
:101B400025E0FE0218CA753AFE78E2E26003122729
:101B5000332042030208FAC242C2AFD2AED2BED292
:101B6000AF0208FA010204081020408000010203BD
:101B7000040002030400010377115E5B396B6F51AF
:101B80007F7B77115E5B396B6F517F7B77115E5B7B
:101B9000396B6F517F7B77115E5B396B6F517F7B48
:101BA00077115E5B396B6F517F7B77115E5B396BB1
:101BB0006F517F7B77115E5B396B6F517F7B771144
:101BC0005E5B396B6F517F7B77115E5B396B6F5159
:101BD0007F7B77115E5B396B6F517F7B77115E5B2B
:101BE000396B6F517F7B77115E5B396B6F517F7BF8
:101BF00077115E5B396B6F517F7B77115E5B396B61
:101C00006F517F7B77115E5B396B6F517F7B7711F3
:101C10005E5B396B6F517F7B77115E5B396B6F5108
:101C20007F7B77115E5B396B6F517F7B77115E5BDA
:101C3000396B6F517F7B77115E5B396B6F517F7BA7
:101C400077115E5B396B6F517F7B77115E5B396B10
:101C50006F517F7B77115E5B396B6F517F7B7711A3
:101C60005E5B396B6F517F7B77115E5B396B6F51B8
:101C70007F7B77115E5B396B6F517F7B77115E5B8A
:101C8000396B6F517F7B77115E5B396B6F517F7B57
:101C900077115E5B396B6F517F7B77115E5B396BC0
:101CA0006F517F7B77115E5B396B6F517F7B771153
:101CB0005E5B396B6F517F7B77115E5B396B6F5168
:101CC0007F7B77115E5B396B6F517F7B77115E5B3A
:101CD000396B6F517F7B77115E5B396B6F517F7B07
:101CE00077115E5B396B6F517F7B77115E5B396B70
:101CF0006F517F7B77115E5B396B6F517F7B771103
:101D00005E5B396B6F517F7B77115E5B396B6F5117
:101D10007F7B77115E5B396B6F517F7B77115E5BE9
:101D2000396B6F517F7B77115E5B396B6F517F7BB6
:101D300077115E5B396B6F517F7B77115E5B396B1F
:101D40006F517F7B77115E5B396B6F517F7B7711B2
:101D50005E5B396B6F517F7B77115E5B396B6F51C7
:101D60007F7B77115E5B396B6F517F7B77115E5B99
:101D7000396B6F517F7B77115E5B396B6F517F7B66
:101D800077115E5B396B6F517F7B77115E5B396BCF
:101D90006F517F7B77115E5B396B6F517F7B771162
:101DA0005E5B396B6F517F7B77115E5B396B6F5177
:101DB0007F7B77115E5B396B6F517F7B77115E5B49
:101DC000396B6F517F7B77115E5B396B6F517F7B16
:101DD00077115E5B396B6F517F7B77115E5B396B7F
:101DE0006F517F7B77115E5B396B6F517F7B771112
:101DF0005E5B396B6F517F7B77115E5B396B6F5127
:101E00007F7B77115E5B396B6F517F7B77115E5BF8
:101E1000396B6F517F7B77115E5B396B6F517F7BC5
:101E200077115E5B396B6F517F7B77115E5B396B2E
:101E30006F517F7B77115E5B396B6F517F7B7711C1
:101E40005E5B396B6F517F7B77115E5B396B6F51D6
:101E50007F7B77115E5B396B6F517F7B77115E5BA8
:101E6000396B6F517F7B77115E5B396B6F517F7B75
:101E700077115E5B396B6F517F7B77115E5B396BDE
:101E80006F517F7B77115E5B396B6F517F7B771171
:101E90005E5B396B6F517F7B77115E5B396B6F5186
:101EA0007F7B77115E5B396B6F517F7B77115E5B58
:101EB000396B6F517F7B77115E5B396B6F517F7B25
:101EC00077115E5B396B6F517F7B77115E5B396B8E
:101ED0006F517F7B77115E5B396B6F517F7B771121
:101EE0005E5B396B6F517F7B77115E5B396B6F5136
:101EF0007F7B77115E5B396B6F517F7B77115E5B08
:101F0000396B6F517F7B77115E5B396B6F517F7BD4
:101F100077115E5B396B6F517F7B77115E5B396B3D
:101F20006F517F7B77115E5B396B6F517F7B7711D0
:101F30005E5B396B6F517F7B77115E5B396B6F51E5
:101F40007F7B77115E5B396B6F517F7B77115E5BB7
:101F5000396B6F517F7B77115E5B396B6F517F7B84
:101F6000087B7B7B7B7B7B7B7B7B7B484848484833
:101F70004848484848575757575757575757575E35
:101F80005E5E5E5E5E5E5E5E5E6C6C6C6C6C6C6C0F
:101F90006C6C6C3E3E3E3E3E3E3E3E3E3E3F3F3FD4
:101FA0003F3F3F3F3F3F3F58585858585858585860
:101FB000587F7F7F7F7F7F7F7F7F7F7E7E7E7E7E5D
:101FC0007E7E7E7E7E7B7B7B7B7B7B7B7B7B7B4885
:101FD0004848484848484848485757575757575718
:101FE0005757575E5E5E5E5E5E5E5E5E5E6C6C6CFC
:101FF0006C6C6C6C6C6C6C3E3E3E3E3E3E3E3E3EBF
:102000003E3F3F3F3F3F3F3F3F3F3F585858585864
:1020100058585858587F7F7F7F7F7F7F7F7F7F7E94
:102020007E7E7E7E7E7E7E7E7E7B7B7B7B7B7B7BE5
:102030007B7B7B484848484848484848485757575A
:10204000575757575757575E5E5E5E5E5E5E5E5EE1
:102050005E6C6C6C6C6C6C6C6C6C6C3E3E3E3E3EB4
:102060003E3E3E3E3E3F3F3F3F3F3F3F3F3F3F586C
:102070005858585858585858587F7F7F7F7F7F7FCF
:102080007F7F7F7E7E7E7E7E7E7E7E7E7E7B7B7B76
:102090007B7B7B7B7B7B7B4848484848484848485B
:1020A00048575757575757575757575E5E5E5E5EAC
:1020B0005E5E5E5E5E6C6C6C6C6C6C6C6C6C6C3ED4
:1020C0003E3E3E3E3E3E3E3E3E3F3F3F3F3F3F3F29
:1020D0003F3F3F585858585858585858587F7F7F56
:1020E0007F7F7F7F7F7F7F7E7E7E7E7E7E7E7E7E09
:1020F0007E7B7B7B7B7B7B7B7B7B7B48484848482C
:102100004848484848575757575757575757575EA3
:102110005E5E5E5E5E5E5E5E5E6C6C6C6C6C6C6C7D
:102120006C6C6C3E3E3E3E3E3E3E3E3E3E3F3F3F42
:102130003F3F3F3F3F3F3F585858585858585858CE
:10214000587F7F7F7F7F7F7F7F7F7F7E7E7E7E7ECB
:102150007E7E7E7E7E7B7B7B7B7B7B7B7B7B7B48F3
:102160004848484848484848485757575757575786
:102170005757575E5E5E5E5E5E5E5E5E5E6C6C6C6A
:102180006C6C6C6C6C6C6C3E3E3E3E3E3E3E3E3E2D
:102190003E3F3F3F3F3F3F3F3F3F3F5858585858D3
:1021A00058585858587F7F7F7F7F7F7F7F7F7F7E03
:1021B0007E7E7E7E7E7E7E7E7E7B7B7B7B7B7B7B54
:1021C0007B7B7B48484848484848484848575757C9
:1021D000575757575757575E5E5E5E5E5E5E5E5E50
:1021E0005E6C6C6C6C6C6C6C6C6C6C3E3E3E3E3E23
:1021F0003E3E3E3E3E3F3F3F3F3F3F3F3F3F3F58DB
:102200005858585858585858587F7F7F7F7F7F7F3D
:102210007F7F7F7E7E7E7E7E7E7E7E7E7E7B7B7BE4
:102220007B7B7B7B7B7B7B484848484848484848C9
:1022300048575757575757575757575E5E5E5E5E1A
:102240005E5E5E5E5E6C6C6C6C6C6C6C6C6C6C3E42
:102250003E3E3E3E3E3E3E3E3E3F3F3F3F3F3F3F97
:102260003F3F3F585858585858585858587F7F7FC4
:102270007F7F7F7F7F7F7F7E7E7E7E7E7E7E7E7E77
:102280007E7B7B7B7B7B7B7B7B7B7B48484848489A
:102290004848484848575757575757575757575E12
:1022A0005E5E5E5E5E5E5E5E5E6C6C6C6C6C6C6CEC
:1022B0006C6C6C3E3E3E3E3E3E3E3E3E3E3F3F3FB1
:1022C0003F3F3F3F3F3F3F5858585858585858583D
:1022D000587F7F7F7F7F7F7F7F7F7F7E7E7E7E7E3A
:1022E0007E7E7E7E7E7B7B7B7B7B7B7B7B7B7B4862
:1022F00048484848484848484857575757575757F5
:102300005757575E5E5E5E5E5E5E5E5E5E6C6C6CD8
:102310006C6C6C6C6C6C6C3E3E3E3E3E3E3E3E3E9B
:102320003E3F3F3F3F3F3F3F3F3F3F585858585841
:1023300058585858587F7F7F7F7F7F7F7F7F7F7E71
:102340007E7E7E7E7E7E7E7E7E047E7E7E7E7E7E27
:102350007E7E7E7E7E7E7E7E7E7E7E7E7E7E7E7E9D
:102360007E7E7E7E7E7E7E7E7E7E7E7E7E7E7E7E8D
:102370007E7E7E7E7E7E7E7E7E7E7E7E7E7E7E7E7D
:102380007E7E7E7E7E7E7E7E7E7E7E7E7E7E7E7E6D
:102390007E7E7E7E7E7E7E7E7E7E7E7E7E7E7E7E5D
:1023A0007E7E7E7E7E7E7E7E7E7E7E7E7E7E181819
:1023B000181818181818181818181818181818189D
:1023C000181818181818181818181818181818188D
:1023D000181818181818181818181818181818187D
:1023E000181818181818181818181818181818186D
:1023F000181818181818181818181818181818185D
:10240000181818181818181818181818181818184C
:1024100018186B6B6B6B6B6B6B6B6B6B6B6B6B6BB2
:102420006B6B6B6B6B6B6B6B6B6B6B6B6B6B6B6BFC
:102430006B6B6B6B6B6B6B6B6B6B6B6B6B6B6B6BEC
:102440006B6B6B6B6B6B6B6B6B6B6B6B6B6B6B6BDC
:102450006B6B6B6B6B6B6B6B6B6B6B6B6B6B6B6BCC
:102460006B6B6B6B6B6B6B6B6B6B6B6B6B6B6B6BBC
:102470006B6B6B6B6B6B5B5B5B5B5B5B5B5B5B5B4C
:102480005B5B5B5B5B5B5B5B5B5B5B5B5B5B5B5B9C
:102490005B5B5B5B5B5B5B5B5B5B5B5B5B5B5B5B8C
:1024A0005B5B5B5B5B5B5B5B5B5B5B5B5B5B5B5B7C
:1024B0005B5B5B5B5B5B5B5B5B5B5B5B5B5B5B5B6C
:1024C0005B5B5B5B5B5B5B5B5B5B5B5B5B5B5B5B5C
:1024D0005B5B5B5B5B5B5B5B5B5B1D1D1D1D1D1DC0
:1024E0001D1D1D1D1D1D1D1D1D1D1D1D1D1D1D1D1C
:1024F0001D1D1D1D1D1D1D1D1D1D1D1D1D1D1D1D0C
:102500001D1D1D1D1D1D1D1D1D1D1D1D1D1D1D1DFB
:102510001D1D1D1D1D1D1D1D1D1D1D1D1D1D1D1DEB
:102520001D1D1D1D1D1D1D1D1D1D1D1D1D1D1D1DDB
:102530001D1D1D1D1D1D1D1D1D1D1D1D1D1D575757
:10254000575757575757575757575757575757571B
:10255000575757575757575757575757575757570B
:1025600057575757575757575757575757575757FB
:1025700057575757575757575757575757575757EB
:1025800057575757575757575757575757575757DB
:1025900057575757575757575757575757575757CB
:1025A00057577777777777777777777777777777FB
:1025B00077777777777777777777777777777777AB
:1025C000777777777777777777777777777777779B
:1025D000777777777777777777777777777777778B
:1025E000777777777777777777777777777777777B
:1025F000777777777777777777777777777777776B
:102600007777777777771A1A1A1A1A1A1A1A1A1AFC
:102610001A1A1A1A1A1A1A1A1A1A1A1A1A1A1A1A1A
:102620001A1A1A1A1A1A1A1A1A1A1A1A1A1A1A1A0A
:102630001A1A1A1A1A1A1A1A1A1A1A1A1A1A1A1AFA
:102640001A1A1A1A1A1A1A1A1A1A1A1A1A1A1A1AEA
:102650001A1A1A1A1A1A1A1A1A1A1A1A1A1A1A1ADA
:102660001A1A1A1A1A1A1A1A1A1A7F7F7F7F7F7F6C
:102670007F7F7F7F7F7F7F7F7F7F7F7F7F7F7F7F6A
:102680007F7F7F7F7F7F7F7F7F7F7F7F7F7F7F7F5A
:102690007F7F7F7F7F7F7F7F7F7F7F7F7F7F7F7F4A
:1026A0007F7F7F7F7F7F7F7F7F7F7F7F7F7F7F7F3A
:1026B0007F7F7F7F7F7F7F7F7F7F7F7F7F7F7F7F2A
:1026C0007F7F7F7F7F7F7F7F7F7F7F7F7F7F5F5F5A
:1026D0005F5F5F5F5F5F5F5F5F5F5F5F5F5F5F5F0A
:1026E0005F5F5F5F5F5F5F5F5F5F5F5F5F5F5F5FFA
:1026F0005F5F5F5F5F5F5F5F5F5F5F5F5F5F5F5FEA
:102700005F5F5F5F5F5F5F5F5F5F5F5F5F5F5F5FD9
:102710005F5F5F5F5F5F5F5F5F5F5F5F5F5F5F5FC9
:102720005F5F5F5F5F5F5F5F5F5F5F5F5F5F5F5FB9
:102730005F5F0178B4760375660F7583F778E3E21F
:10274000F582E22410F2C394F040037422F2AF82C7
:10275000AE83E078B6F60582AF82E054F008F674F6
:10276000032582F582E0C4540F46F6E6540FFFC3FA
:102770009409501DAD82AC8374F0F008EF28F56524
:10278000E8C3956550140582AF82AE83E0F60880F9
:10279000EFD566A978E2E214F22278E2E214F27848
:1027A00080E220E30302285C78B6E6FF64037052FF
:1027B00078B9E6FE18E6FD24D9F8EEF278BAE6FE1E
:1027C000ED25E025E024ADF8EEF278BBE6FEED2540
:1027D000E025E024AEF8EEF278BCE6FEED25E0253B
:1027E000E024AFF8EEF278BDE6FEED25E025E0242A
:1027F000B0F8EEF27401A805088002C333D8FC4299
:102800005C22EF6404703B78BAE6FF78B8E6FE25F8
:10281000E025E0245AF8EFF278BBE6FFEE25E0254C
:10282000E0245BF8EFF278BCE6FFEE25E025E0243B
:102830005CF8EFF278BDE6FFEE25E025E0245D02CE
:102840002E4A78B6E6B4051478BAE6FE18E67C009F
:102850002400FFEC3EFE18E6FD023DE878CAE6FFE4
:1028600044C0FE78B6E6FDB5061708E67013EF70B3
:1028700003022E9478CAE6F52E78A8E4F20804F252
:1028800022ED6435600302296F78B7E6FFB40115C5
:1028900008E6B40D1090000574FFF0A3F0C2EBD26F
:1028A000E9D2EA80F078B8E6FE64076004EEB40886
:1028B0000BE4F551C244C22C75358A22EE7006C273
:1028C00025C248C228EEB40104D225C248EE6402F3
:1028D0006005EE64037073E4F556F557C225D248DF
:1028E000F530F52E300803432E01301003432E023D
:1028F000300903432E04301103432E08300A0343EA
:102900002E10301203432E20300B03432E40301381
:1029100003432E80300C0343300130140343300254
:10292000300D03433004301503433008300E0343A9
:102930003010301603433020300F0343304030173F
:1029400003433080852E37853039EE640B600302F7
:102950002E94EF64026003022E94D22F78B9E6FF22
:1029600030E102D236EF20E003022E94D2392278F1
:10297000B6E6FFB4451478B8E664056003022E9409
:10298000C244C22C75358AF55122EF641D600302E2
:102990002B3778B7E66402702A08E6FF78CA6660CB
:1029A00008EF64636003022E9412409378C9E6FF37
:1029B000F47003022E9478D8EFF278B9E678CDF26D
:1029C000D2292278B7E664036003022AF679B8E7D1
:1029D00078CA666003022E9478B9E6700A08E6D3D6
:1029E000943F4003022E9412409378C9E6F470039A
:1029F000022E9478C9E6FF78D8F278B9E678CDF25D
:102A000078BAE678CEF2EFB41B12E278ACF260044A
:102A1000E2B4FF0878AC7482F278CEF278C9E6FFAF
:102A2000B41C1478CEE2787DF26004E2B4FF08783A
:102A30007D7488F278CEF2EFB41D1578CEE278D8A6
:102A4000F66004E6B4FF0978D8760178CE7401F216
:102A500078C9E6FFC394134054EF941B504FEF2402
:102A6000EDFF7401A807088002C333D8FC78C8F6CC
:102A7000E478C1F608760178C1E6FFC39408502DCA
:102A800079BAE70856600C74AB2FF978C8E6F457AA
:102A9000F7801078C1E624ABF8C000F9E778C846A3
:102AA000D000F678C10608E625E0F680CA78C9E6C7
:102AB000FFC3940B4011EF9413500C78CEE2FF78D3
:102AC000C9E62402F8EFF278C9E6FFC3941E40116C
:102AD000EF9426500C78CEE2FF78C9E62471F8EF27
:102AE000F278C9E6B4260578CEE208F278CEE2F4B0
:102AF000787BF2D2302278B7E664046003022E9429
:102B000078B8E6F56678BA666003022E9478B9E67E
:102B1000F56578BB666003022E94E566F465656032
:102B200003022E94E566600878CAE66003022E94DC
:102B300078CAA666D2232278B8E66463705878B65D
:102B4000E6FF64196005EF641C703FE4F56FF570F3
:102B5000F571F572F573F574F575F5767898F208F8
:102B6000F208F208F208F208F208F208F208F20895
:102B7000F208F208F208F208F208F208F2FE7F0802
:102B8000FD7BFE7AF8790012448278B6E6B4190427
:102B9000D23D8002C23D79B8E778CA666003022E52
:102BA0009478B6E6FF64187003022E94EF641F70E9
:102BB0002D787CF278B7E664056003022E9478B92C
:102BC000E6FF78BB666003022E9418E6F46F60039C
:102BD000022E947880EFF278BCE678CBF62278B6B5
:102BE000E6FFB41904755CFF22EF641A702B78B706
:102BF000E6C4135407FF7401A807088002C333D842
:102C0000FCF4F566525CE52F64806005787AE52F68
:102C1000F2752F80E56652552278B6E6641B600394
:102C2000022CB4787CF278B7E6C4135407F5662416
:102C3000E4F8E4F2740D2566F8E2C39464503E783B
:102C4000B9E6FFB4041E746F2566F8E4F674002537
:102C500066F8E4F274402566F582E434F9F583748D
:102C60000AF08019746F2566F8EFF674002566F88F
:102C7000EFF278CFE2D394004003123B8178B7E6BD
:102C8000540F64027003022E9478BAE6FF5407FED4
:102C90007401A806088002C333D8FCF566EF30E360
:102CA00009787BE64566F6022E75E566F4787B5674
:102CB000F6022E7578B6E6641C6003022E4E787C10
:102CC000F278B7E6FFC4135407F566EF540F6403B8
:102CD0006003022D9D740D2566F8E2C394644003E1
:102CE000022E9478B9E6FF746F2566F8EFF6FF744C
:102CF000002566F8EFF278BAE6FF74E42566F8EF8F
:102D0000F274E42566F8E2FD33502C74017E00A8CD
:102D100066088005C333CE33CED8F9FFE521FBEF3B
:102D20005B24FF5012ED5407FF746F2566F8EFF631
:102D300074002566F8EFF274E42566F8E2FDA2E679
:102D4000502C74017E00A866088005C333CE33CEB4
:102D5000D8F9FFE522FBEF5B24FF5012ED5407FF8B
:102D6000746F2566F8EFF674002566F8EFF2746F5D
:102D70002566F8E6B40418E4F674002566F8E4F273
:102D800074402566F582E434F9F583740AF02278FC
:102D9000CFE2D394005003022E94022E7574E425E2
:102DA00066F8E4F278B9E6FF64637003022E947863
:102DB000B7E6C4135407F566FE7401A8060880023E
:102DC000C333D8FCFE425C740D2566F8E2C39464FC
:102DD0004003022E94EF547FFF6404702878B9E614
:102DE00020E722746F2566F8E4F674002566F8E49F
:102DF000F274402566F582E434F9F583740AF0EE46
:102E0000F4525C8019746F2566F8EFF6740025663D
:102E1000F8EFF278CFE2D394004003123B8178B907
:102E2000E630E770787AE2F52F303D6874EC25667D
:102E3000F8E2600B746F2566F8E6FF7498800974F9
:102E40006F2566F8E6FF74A02566F8EFF22278B6E3
:102E5000E6641E703F787CF278B7E6540FF566B4EE
:102E6000021678B9E6FF7401A807088002C333D8B8
:102E7000FC787B66F6023B8178B9E6900002F008A8
:102E8000E6A3F0E566B4050CC23408E6900000F055
:102E900008E6A3F022C000C001C002C092759205EE
:102EA000E4C54EF4D3340FFAF9FF70030230DE7537
:102EB0008200789B76000876000876000876000885
:102EC0007600087600087600087600087600087616
:102ED000000876000876000876000876000876007C
:102EE000087600789BE0FE541126F608EE03FE54A7
:102EF0001126F608EE03FE541126F608EE035411CF
:102F000026F6080582E0FE541126F608EE03FE546C
:102F10001126F608EE03FE541126F608EE035411AE
:102F200026F6080582E0FE541126F608EE03FE544C
:102F30001126F608EE03FE541126F608EE0354118E
:102F400026F6080582E0FE541126F608EE03FE542C
:102F50001126F608EE03FE541126F608EE0354116E
:102F600026F6080582DA028003022EE3789BE9C385
:102F700013FA797D7700E6540FD39AC792E3C7E43A
:102F8000C608C4540FD39AC792E703C7E6540FD3B9
:102F90009AC792E3C7E4C608C4540FD39AC792E70E
:102FA00003C7E6540FD39AC792E3C7E4C608C454D4
:102FB0000FD39AC792E703C7E6540FD39AC792E399
:102FC000C7E4C608C4540FD39AC792E7C7797E777F
:102FD00000E6540FD39AC792E3C7E4C608C4540F5F
:102FE000D39AC792E703C7E6540FD39AC792E3C7B1
:102FF000E4C608C4540FD39AC792E703C7E6540F38
:10300000D39AC792E3C7E4C608C4540FD39AC792B1
:10301000E703C7E6540FD39AC792E3C7E4C608C4D0
:10302000540FD39AC792E7C779817700E6540FD33C
:103030009AC792E3C7E4C608C4540FD39AC792E76D
:1030400003C7E6540FD39AC792E3C7E4C608C45433
:103050000FD39AC792E703C7E6540FD39AC792E3F8
:10306000C7E4C608C4540FD39AC792E703C7E6540F
:103070000FD39AC792E3C7E4C608C4540FD39AC7C4
:1030800092E7C779827700E6540FD39AC792E3C7D5
:10309000E4C608C4540FD39AC792E703C7E6540F97
:1030A000D39AC792E3C7E4C608C4540FD39AC79211
:1030B000E703C7E6540FD39AC792E3C7E4C608C430
:1030C000540FD39AC792E703C7E6540FD39AC79217
:1030D000E3C7E4C608C4540FD39AC792E7C7758202
:1030E00000754E0FD092D002D001D00022C0E0C0B7
:1030F000D075D00820271485C638E5C7700DE5388F
:103100009464500AD2BDD0D0D0E0327538FFC227C7
:10311000C295D295200419E53894BE9202BC001ED7
:103120002002677D07C207D204D2337F000231B488
:10313000E53894B4500685385E0231C8806E30029E
:103140005C1CE52B6044D52B41755100E778835614
:10315000F54FC28EC28FD22A85FF8D304502158D64
:1031600078D7E6F4F58BC2477464309303D5E0FA60
:10317000209305D5E0FA8006309309D5E0FAC22AFB
:103180007C0A8006D28EC2C8C2BDD0D0D0E032BA8E
:1031900000047B008022DA20752B007B007C0A80F3
:1031A000E9EE33FE50E46FFFD20580DE7C0C1007A1
:1031B000323005EDDD5480D7C3740C9CFC740A9C3E
:1031C0005001E4FCC20480C2DC04C20480BC1007CD
:1031D000E73005CDC205A892759204EF938892D28C
:1031E0000780A7752DFFBB0017D22D7A00752B0124
:1031F00078847987B60A0F752B0379AB740A80C37C
:10320000DB04D22D7A00740A80B9E54E6029154E90
:10321000E4C591F52B7800A992759205E2F00805B6
:1032200082E2F0080582E2F0080582E2F00582857C
:103230002B918992752B00C2057E01855D54303338
:103240002DC233204428D247758DFB758BD5D28E85
:10325000053CE53CB4131585FFF878CCE6F4A8925C
:10326000759203F08892753C0002318AC22C0231BB
:103270008A000101020102020301020203020303A8
:10328000040102020302030304020303040304040F
:1032900005010202030203030402030304030404FE
:1032A00005020303040304040503040405040505DF
:1032B00006010202030203030402030304030404DD
:1032C00005020303040304040503040405040505BF
:1032D00006020303040304040503040405040505AE
:1032E000060304040504050506040505060506068F
:1032F000070102020302030304020303040304049C
:10330000050203030403040405030404050405057E
:10331000060203030403040405030404050405056D
:10332000060304040504050506040505060506064E
:10333000070203030403040405030404050405054C
:10334000060304040504050506040505060506062E
:10335000070304040504050506040505060506061D
:1033600007040505060506060705060607060707FE
:10337000087B2E756737756804756908756A027F62
:10338000018F648D658B66E56AF4F56BE564787F83
:1033900030E00F7410F278817420F278857440F276
:1033A000800C7401F2788104F278857404F2E56B84
:1033B000523B746F2564F8E6B4041B202C030237DB
:1033C0006B788D7402F2788204F278AA7406F2782F
:1033D000897414F28014788D740AF27882741EF263
:1033E00078AA7412F2788974C8F2E556556A602991
:1033F00074922564F56CF816E6600302376BE56B92
:103400005256E56A4257A865A9007885E2F457F755
:1034100078AAE224FDA86CF622A9657885E25760B7
:103420005BE557556A60127889E2FF74922564F86B
:10343000A607E56A425602376774922564F56CF870
:10344000060606A90078AAE2FFE7C39F50030237E9
:103450006B7889E2A86CF678B57603E56A42564245
:103460005C4255A866E64568FFF6E569F45FF6A894
:1034700067E64569FFF6E568F45FF6227492256415
:10348000F56CF8E6600116A965787FE257700302D3
:103490003579743E2564F56CE521556A60067882BD
:1034A000E2A86CF6A96C788DE2FFE7C39F400302A7
:1034B00035D2A86C06E6C39F50030235D2E52F64CF
:1034C000806006A86C160235D274E42564F56D742C
:1034D0006F2564F56EA866E64568F6A867E6456858
:1034E000F6E56B525778B57603E56A4221425C42B5
:1034F00055E4F52F7882E2A86CF6A86DE2FF30E77C
:10350000055407A86EF6E522556A604C748F256451
:10351000F8E2F55B30E313A86EE64480FF74002503
:1035200064F8EFF2A86EE4F6802EE55B30E413A8B1
:103530006EE64480FF74002564F8EFF2A86E760111
:103540008016E55B30E511A86EE64480FF74002527
:1035500064F8EFF2A86E760278CFE2D394004003CD
:10356000123B81303D6C74982564F8E2A86EF674C5
:10357000EC2564F87401F28059743E2564F56CE51D
:1035800021556A7003A86CF6A86CE6604516E670D3
:1035900041E56B52575221A866E6FFE568F4FE5FED
:1035A000F6A867E65EF678B57603E56A425C4255B2
:1035B0005522701E74002564F8E230E715547FFF31
:1035C000746F2564F8A60778CFE2D3940040031205
:1035D0003B81A9657881E25770030236C2744625A3
:1035E00064F56CE522556A600508E2A86CF6A96CE2
:1035F000788DE2FFE7C39F400302371BA86C06E605
:10360000C39F500302371BE52F64806006A86C1629
:1036100002371B74E42564F56D746F2564F56EE55F
:103620006B5257A866E64569F6A867E64569F678DD
:10363000B57603E56A4222425C4255752F087882CE
:10364000E2A86CF6A86DE2FF30E6055407A86EF616
:10365000E521556A604C748F2564F8E2F55B30E033
:1036600013A86EE64480FF74002564F8EFF2A86E9C
:10367000E4F6802EE55B30E113A86EE64480FF742B
:10368000002564F8EFF2A86E76018016E55B30E263
:1036900011A86EE64480FF74002564F8EFF2A86E6E
:1036A000760278CFE2D394004003123B81303D6B29
:1036B00074A02564F8E2A86EF674EC2564F8E4F2D0
:1036C000805974462564F56CE522556A7003A86C30
:1036D000F6A86CE6604516E67041E56B525752223B
:1036E000A866E6FFE569F4FE5FF6A867E65EF67891
:1036F000B57603E56A425C42555521701E7400257B
:1037000064F8E230E715547FFF746F2564F8A6076C
:1037100078CFE2D394004003123B81E557556A60AD
:103720004AE56A425C42555521A866600CE6456848
:10373000F6A867E64568F6800DE6FFE568F4FE5FEB
:10374000F6A867E65EF6E522556AA866600CE645CF
:1037500069F6A867E64569F6800DE6FFE569F4FEBF
:103760005FF6A867E65EF6E56B525722C0E0C083BD
:10377000C082C0D075D010202A03023870C28E7566
:103780008DFF789AE6F4F58BD28E202E0D20440A18
:10379000E54FF4900004F0854FF830386AAF8CEFB5
:1037A000F4FFEFFEAD8AEDF4FDE4F4FCE42D78883F
:1037B000F2EE3C18F2C238D246208D0DE2FE08E24D
:1037C000FFD3941EEE9400500A78877408F20874B0
:1037D00054802FC3EF9454EE9408401B7888E22461
:1037E000ACF218E234F7F2D221C222C28C758CF707
:1037F000758AABD28C8010C374549F7888F2740899
:103800009E18F2D222C2217884E6B40A1C055174B3
:10381000AB2551F8E6F54F7883E6524FE551640940
:1038200060030239F208F6801A055174872551F8B1
:10383000E6F54F7883E6524FE5516407600302399D
:10384000F20806C28EC22A755100D23BC246C2227D
:10385000C221D23EC2C2C2C3303904D2BAD220750C
:103860002AFF752DFFC2C4C2C5D2C8D2BD0239F22B
:10387000C28E202E4020443D30472F900000E0F4BF
:103880007877F6A3E0F408F6A3E0F408F6A3E0F4F2
:1038900008F685573B75F8FF78D6E6F4A3F0E53CCB
:1038A00060030239F2D22C0239F275F8FF78D6E6BD
:1038B000F4900004F0C2C2C2C3303E05303902D2D7
:1038C000BAC2BB3090021552E55264187020C23162
:1038D000D243787FF6302007C220F5530239F2E553
:1038E0005364106005E553B41402D2418027E552B9
:1038F00064197029C231D243787F06E6B405027696
:1039000000302004C220800FE55364106005E553A9
:10391000B41402D241D2287553000239F230310377
:103920000239F2E552C394084004D24B8002C24BE4
:10393000E553B4140040030239ED903941F82828CA
:103940007302397D02398502398D02399502399D1C
:103950000239A50239AD0239B50239BD0239BD02BD
:1039600039BD0239BD0239BD0239BD0239C1023942
:10397000E30239BD0239BD0239BD0239BDA24B9205
:103980001F0553806DA24B921E05538065A24B927A
:103990001D0553805DA24B921C05538055A24B928E
:1039A0001B0553804DA24B921A05538045A24B92A2
:1039B000190553803DA24B9218055380350553805D
:1039C00031D2EF055375F8FF203B27D23AE53C642E
:1039D00013701F202E1C20441978CCE6F4900004AC
:1039E000F0800FC2EF055380090553800575530021
:1039F000D231D0D0D082D083D0E032C0E0C083C0FA
:103A000082C0D075D018C28C30214A30462F900029
:103A100000E0F47877F6A3E0F408F6A3E0F408F603
:103A2000A3E0F408F685573B75F8FF78D6E6F44531
:103A300057A3F0E557F4788356F6752B00C246C2BB
:103A4000217887E2FC08E2FDECF4F58CEDF4F58AD0
:103A5000D28C023B78D22B202403023AF2C2247586
:103A6000FA01E53AD39444500878ABE2F4900007A9
:103A7000F0E53AC39444506F900000E0F531A3E0C4
:103A8000F532A3E0F533A3E0F534E4FFE53130E3AC
:103A9000010FE53130E703431F02E53230E3034312
:103AA0001F04E53230E703431F08E53330E30343E7
:103AB0001F10E53330E703431F20E53430E30343B1
:103AC0001F40E53430E703431F807416253AF8EFB2
:103AD000F2E53AC39404500B7408253AF8E278AB47
:103AE000F2800478ABEFF2E53AC394465056053ABB
:103AF0008052E53AB4FE1075FA00753AFF78ABE4EF
:103B0000F2900007F08037E53AB4FF05753A00807F
:103B10000EE53AD39444500778ABE2900007F07575
:103B2000FA0000000000000000000000000000009B
:103B3000000000000000000000000075FA01D2241F
:103B4000D232D242302229C28C7887E2FC08E2FDD0
:103B5000ECF4F58CEDF4F58AD28C18E2FE08E2FF65
:103B6000C374059FF2740D9E18F2C222D221800800
:103B7000758CF2758AFAD28CD0D0D082D083D0E006
:103B800032E4FF78CFE2FE30E01BE56F543F600E79
:103B900024FC600A24A1601B24607004800D801046
:103BA000430703800E787BE630E00543070280037D
:103BB000430701EE30E11BE570543F600E24FC60CA
:103BC0000A24A1601B24607004800D801043070C40
:103BD000800E787BE630E105430708800343070445
:103BE00078CFE2FE30E21BE571543F600E24FC60AA
:103BF0000A24A1601B24607004800D8010430730EC
:103C0000800E787BE630E2054307208003430710EF
:103C1000EE30E31BE572543F600E24FC600A24A1E1
:103C2000601B24607004800D80104307C0800E78F4
:103C30007BE630E3054307808003430740900002A2
:103C4000EFF0E4FF78CFE2FE30E41BE573543F6011
:103C50000E24FC600A24A1601B24607004800D8087
:103C600010430703800E787BE630E40543070280AB
:103C700003430701EE30E51BE574543F600E24FC5E
:103C8000600A24A1601B24607004800D801043072B
:103C90000C800E787BE630E5054307088003430778
:103CA0000478CFE2FE30E61BE575543F600E24FC3D
:103CB000600A24A1601B24607004800D80104307FB
:103CC00030800E787BE630E605430720800343070B
:103CD00010EE30E71BE576543F600E24FC600A24AA
:103CE000A1601B24607004800D80104307C0800E0B
:103CF000787BE630E7054307808003430740900068
:103D000003EFF022FF7D018F648D65E565D3940498
:103D10004003023DE77DC0AB65AF6412439950F5A7
:103D2000E564242AFF7DC4AB6512439950F2E56433
:103D30002454FF7D8EAB6512439950F2E4F566E59D
:103D400066C395654003023DE774C42566F974C0F7
:103D50002566F8E6FF677021748E2566F8E66F70B9
:103D600003023DE2E56425662454FF74C02566FD28
:103D70007B0112421C406B80EB748E2566F8E6FFD7
:103D800074C02566F8E66F701E74C42566F8EF6689
:103D90006050E5642566242AFF748E2566FD7B014C
:103DA00012421C403D80EB74C42566F8E6FF748E19
:103DB0002566F8E6FE6F702374C02566F8EE66602F
:103DC0002174C02566F8A607E5642566FF748E2574
:103DD00066FD7B0112421C400980ED74C02566F827
:103DE000E4F60566023D3F2222C2AF900007EDF0E7
:103DF0000074FFF0D2AF7C0174782FF582741B3E03
:103E0000F583E493FBEC601E5B600FC2AF9000078C
:103E1000EDF00074FFF0D2AF800612452774FFF07A
:103E2000EC25E0FC80DF7C01D3EF9409EE940040A8
:103E30001174612FF582741F3EF583E4934480FB77
:103E400080027B80EC601E5B600FC2AF900007EDCC
:103E5000F00074FFF0D2AF800612452774FFF0EC3B
:103E600025E0FC80DF7C01C3EF9464EE9400500FEA
:103E7000E4FB12452774FFF000000BBB18F422741A
:103E80004A2FF58274233EF583E493FBEC601E5BBE
:103E9000600FC2AF900007EDF00074FFF0D2AF806A
:103EA0000612452774FFF0EC25E0FC80DFE4FB12EE
:103EB000452774FFF000000BBB10F42278CAE6FF20
:103EC00078C5F6EFF4787BF27DC57B017F068F64C1
:103ED0008D658B66A965787BE2F4677023E566647F
:103EE00001600EE566D394014016788CE2F4B56467
:103EF0000F7897E566F2FBAD65AF6412421C50F196
:103F0000A965787BE2F4677027E5666401600EE5D9
:103F100066D39401401A788CE2F4B564137897E57F
:103F200066F2E564242AFFAB66AD6512421C50EDD3
:103F3000A965787BE2F4677027E5666401600EE5A9
:103F400066D39401401A788CE2F4B564137897E54F
:103F500066F2E5642454FFAB66AD6512421C50ED79
:103F60002275B12075E8F178FEE4F6D8FD90F800EE
:103F70007F007E08E4F0A3DFFCDEFA75A0F875810F
:103F8000E4023FBF020100E493A3F8E493A34003DB
:103F9000F68001F208DFF48029E493A3F8540724A3
:103FA0000CC8C333C4540F4420C8834004F4568063
:103FB0000146F6DFE4800B010204081020408090E7
:103FC0004351E47E019360BCA3FF543F30E50954A4
:103FD0001FFEE493A360010ECF54C025E060A8400B
:103FE000B8E493A3FAE493A3F8E493A3C8C582C802
:103FF000CAC583CAF0A3C8C582C8CAC583CADFE9D7
:10400000DEE780BEC0E0C083C082C0D075D018900B
:10401000F701AF82AE83E030E710204C0DD24C7533
:1040200082007403F0740AF08060C24C758202AEA4
:1040300083E0FFC394024052EFD39410504CBF0270
:10404000047F0F80021F1FEFC454F0F582AE83740B
:1040500041F078E2E204F2E2B40108E58254F0446F
:104060000208F274112582F582C394F04003758230
:1040700021AF82AE837455F074052582F58274F009
:10408000F074FA2582F5827499F0D0D0D082D08372
:10409000D0E03278C976FF78B9E6FF700578C97646
:1040A0000622EFB4110578C9761B22EFB412057809
:1040B000C9761C22EFB4130578C9761D22EFC3948C
:1040C000014007EF94095002801E78B9E6FFC394BF
:1040D000144007EF941C5002800E78B9E6FFC39499
:1040E00009400CEF94115007EF240A78C9F62278A2
:1040F000B9E6FFB41C0578C9762622EFB41D057811
:10410000C9762722EFB41E0578C9762822EFB41F9E
:104110000578C9762922EFB4200478C9762A22903E
:10412000F7007443F090F70474C3F0A3741CF0A379
:10413000E4F0A3F090F70CF0A3F090F7167408F0F9
:1041400090F7117455F090F7107495F090F7207473
:1041500040F090F730F090F740F090F750F090F783
:1041600060F090F770F090F780F090F790F090F793
:10417000A0F090F7B0F090F7C0F090F7D0F090F783
:10418000E07499F0A37455F090F7E67480F090F71E
:10419000F07440F090F700740AF078E374D2F222E1
:1041A000E678C9F6E4F890F711E0543064207028FE
:1041B000900001E0FF900000E02FFF900002E02F50
:1041C000F56408E8D394B440DD204C4FD24C90F70E
:1041D000007403F0740AF02278C0E690F712F00839
:1041E000E6FF54E0A3F0EFC454F0440890F716F053
:1041F000E6540FF5640828F564E8C39564500B0590
:1042000082E6AD82AC83F00880EF758211AE8374D4
:1042100065F0788A744BF278B57603228F678D68E3
:104220008B69C24978DAA6691245377FA01244D952
:104230005059AF671244D95052D249AF691569EF4E
:104240006049A968787BE2F467700778DAE6656907
:10425000600778DAE66569601F78DAE6FF64016076
:104260000DEFD394014011788CE2F4B5670A78978A
:10427000E2FFE569C39F4004C249800FAF6805684B
:10428000A807E6FF1244D940B2C2491245147897F4
:104290007401F2A24922C0E0C083C082C0D075D0B0
:1042A00010758B37758DFF755201C2BAC2C3303A93
:1042B0003EC23AE53CB41307753C00D22C8004059D
:1042C0003CC22CC2B5D226900000E0F47877F6A369
:1042D000E0F408F6A3E0F408F6A3E0F408F6202ED4
:1042E0000C20440975F8FF78D6E6F4A3F0D2B53077
:1042F0003E04D2BBD28ED0D0D082D083D0E032C0A8
:10430000E0C083C082C0D075D010E58BD3946940E3
:1043100037C28E0552E552B41219758B37758DFF71
:10432000202E2320442075F8FF7880E6F4900004C6
:10433000F08013E55264106007E552B4110280006A
:10434000758B37758DFFD28ED0D0D082D083D0E0E0
:1043500032C1BEC141C13BC144C1AEC1B1C1B4C192
:1043600027C137818A4B012F80817A808283820026
:10437000818682015E82014E40013AFE818B0001FE
:104380002B00C126015D09817E00818C008197018F
:10439000C12B818E00013B00008F678D688B69C245
:1043A000491245377FA01244D9502DAF671244D926
:1043B00050261245377FA11244D9501CD249AF690B
:1043C0001569EF6013E56924FF924A12441CAE6838
:1043D0000568A806A60780E6124514A2492222EE27
:1043E000C3940F5010900007EFF012452C74FFF0AB
:1043F00000000E80EA12452CC2AF900007EFF000DB
:1044000074FFF0D2AF12452CE4FE900007EFF012DB
:10441000452C74FFF000000EBE18EF227F08C2AFDB
:10442000D296E4FED29400A296E4334206C294EF00
:10443000D394014004EE25E0FEDFE9304A03C38057
:1044400001D3929600D29400C294D2AFAF0622C09C
:10445000E0C0D075D0087520007C0AE59275920303
:1044600090000475920490327175920590F9007570
:104470009206900000F592752DFF754E0FD0D0D0AA
:10448000E022EF4E6012EF60010EEDBB010B89825E
:104490008A83F0A3DFFCDEFA2289F05007F709DFF8
:1044A000FCA9F022BBFEFCF309DFFCA9F022A3F07B
:1044B0007F648F64C232E564601E78E2E2600312BA
:1044C000273330420AC242C2AFD2AED2BED2AF30E0
:1044D00032E4C232156480DE227E08C2AFEF33922E
:1044E00096EF25E0FFD29400C294DEF1D29600D27E
:1044F0009400A296B3924AC294D2AFA24A2222E575
:1045000064C39428500DEF12452874FFF000000595
:104510006480EC227F64C29400C29600D29400D2E0
:1045200096209602DFF022ED900007F000000000D8
:1045300000000000000022C2AFD29600D29400C258
:104540009600C294D2AF22FFFFFFFFFFFFFFFFFFE5
:00000001FF
